:100000000C94D1040C94F9040C94F9040C94F904A4
:100010000C94F9040C94F9040C94F9040C94F9046C
:100020000C94F9040C94F9040C94F9040C94F9045C
:100030000C94F9040C94F9040C94F9040C94F9044C
:100040000C94D3150C94F9040C94A1150C947B1505
:100050000C94F9040C94F9040C94F9040C94F9042C
:100060000C94F9040C94F9042C20226454696D65F5
:10007000223A002C2022696D7050657255223A0098
:100080002C202272656164696E67223A007B2243EC
:10009000223A0020746F2000454550524F4D202DCC
:1000A00020666F726D617474696E6720617265613C
:1000B0002066726F6D20002C2073617665496E7426
:1000C0003D002C206E6F496D70546F75743D003A81
:1000D00020696D70506572556E69743D00434F4ED6
:1000E00046204300534156494E4720474C4F42411A
:1000F0004C20434F4E46494700494E464F3A205305
:10010000617665642063757272656E7420726561D4
:1001100064696E6720746F20454550524F4D2E0024
:100120002C206E4F66667365743D002C206F6666EA
:100130007365743D002C20645365743D002C20775A
:10014000436F756E743D003A20646174613D0049EF
:100150004E464F3A207072696E74696E67207374F0
:100160006F72656420696D70756C736520636F755F
:100170006E746572206F66204300494E464F3A20E8
:10018000726573746F72656420696D70756C7365E8
:1001900020636F756E746572206F662043004E4F4A
:1001A0005448494E4720464F554E44202D20454542
:1001B00050524F4D2061726561207365656D7320EB
:1001C000656D70747920666F7220430064536574A6
:1001D000096F66667365740961646472097743091F
:1001E0006C774309646174610976616C69640074B9
:1001F0007279696E6720746F20726573746F7265AF
:10020000206C61737420696D70756C736573206305
:100210006F756E7420666F72204300494E464F3AE8
:100220002073617665642063757272656E742070E8
:10023000756C73657320636F756E7420746F2045E1
:100240004550524F4D002C20645365743D002C20C6
:100250006F66667365743D002C2077436F756E740E
:100260003D002020646174613D0073746F726543CA
:10027000757272656E74496D70756C7365733A2032
:100280004300736176656420616C6C206461746105
:100290002C20726573657474696E6720696E200026
:1002A00041444452093009310932093309340935CE
:1002B0000936093700454550524F4D2D4461746150
:1002C0003A002C20707772476F6F643D00504F5793
:1002D00045523A20707772437572723D002C20703F
:1002E0007772476F6F643D002C20646562526563CE
:1002F0006F763D002C206465626F756E63653D000E
:10030000434F4E4620474C4F423A20646562756722
:100310006C6576656C3D0020636F6E6669672027AB
:100320006E6F496D70546F75742720696E76616CBD
:1003300069642120446964206E6F7420736176655E
:100340002E005741524E494E473A204300202D205F
:100350006E6F496D70546F75743D00534156494E30
:100360004720430020636F6E66696720276E6F49E0
:100370006D70546F75742720696E76616C696421A5
:1003800020446964206E6F7420736176652E005777
:1003900041524E494E473A204300202D206E6F496E
:1003A0006D70546F75743D00534156494E4720435C
:1003B0000020636F6E6669672027696D70506572F3
:1003C000556E69742720696E76616C6964212044DA
:1003D0006964206E6F7420736176652E00574152F8
:1003E0004E494E473A204300202D20696D705065DC
:1003F00072556E69743D00534156494E4720430083
:10040000554E4B4E4F574E20434F4D4D414E443A63
:100410002027006F7574206F662072616E676520FB
:10042000302D31353030300077436F756E74204396
:1004300000494E464F3A20736574206E65772072EE
:10044000656164696E673A2000494E464F3A2073F1
:100450006574206E657720696D70756C7365733A8D
:100460002000494E464F3A20736574206E65772010
:1004700072656164696E673A20004552524F523A84
:1004800020696E76616C696420646563696D616C76
:100490007320666F722073657420696D7050657289
:1004A000556E69743D00494E464F3A20736574207D
:1004B0006E65772072656164696E673A2000676FC8
:1004C000742076616C696420636F756E7465722048
:1004D0006E756D6265723A20004552524F523A2055
:1004E000696E76616C696420636F756E74657220E5
:1004F0006E756D626572004552524F523A206D69B9
:100500007373696E672076616C696420636F756EC2
:10051000746572206E756D62657200534156494E66
:100520004720434F4E46494700696E76616C6964C7
:1005300020636F6D6D616E6400756E6B6E6F776EAC
:1005400020706172616D657465722027004552529A
:100550004F52202D20696E76616C69642073796E2C
:10056000746178006D697373696E6720636F756E6F
:10057000746572206E756D626572006465626F7578
:100580006E63653A20002C206465626F756E63654A
:100590005265636F763D005245533A20736574206F
:1005A0006465626F756E63653D005245533A207312
:1005B000657420707772476F6F643D00696E766175
:1005C0006C696420636F756E746572206E756D6200
:1005D0006572006D697373696E6720636F756E7401
:1005E0006572206E756D62657200696E76616C6908
:1005F0006420636F756E746572206E756D626572CE
:10060000006D697373696E6720636F756E746572D0
:10061000206E756D6265720044454255472044491D
:100620005341424C454400444542554720454E41C4
:10063000424C45440000000000250028002B00002B
:10064000000000240027002A0020636F6E6669679F
:100650002073617665496E7420697320696E7661D6
:100660006C696420286F7574206F662072616E67F4
:100670006520302D333630302921005741524E4904
:100680004E473A2043002C2073617665496E743DD5
:100690000020636F6E666967206E6F496D70546FDE
:1006A000757420697320696E76616C696420286FA7
:1006B0007574206F662072616E676520302D333649
:1006C00030302921005741524E494E473A204300CD
:1006D0002C206E6F496D70546F75743D0020636FF0
:1006E0006E66696720696D70506572556E69742019
:1006F000697320696E76616C696421005741524EBE
:10070000494E473A204300696D70506572556E69D5
:10071000743D006C6F6164696E6720636F756E7401
:1007200065727320636F6E663A00696E76616C69FC
:10073000642076616C75652073746F7265640070F7
:100740007772476F6F643A2000696E76616C6964F6
:100750002076616C75652073746F726564006465E2
:10076000626F756E6365323A2000696E76616C69FE
:10077000642076616C75652073746F7265640064C3
:1007800065626F756E6365313A2000202D20696EB9
:1007900076616C69642076616C75652073746F7224
:1007A0006564006A736F6E3A2000202D20696E76B2
:1007B000616C69642076616C75652073746F726515
:1007C000640064656275676C6576656C3A20006CE0
:1007D0006F6164696E6720676C6F62616C20636F24
:1007E0006E663A00494E464F3A20726573746F72D6
:1007F00065642072656164696E67206F66204300DE
:100800004552524F523A204641494C454420746F5C
:1008100020726573746F7265206C617374207265E9
:100820006164696E67206F66204300494E464F3A07
:100830002073746F7265642072656164696E67739A
:10084000203220616E6420332061726520657175ED
:10085000616C00494E464F3A2073746F7265642094
:1008600072656164696E6773203120616E64203344
:100870002061726520657175616C00494E464F3A82
:100880002073746F7265642072656164696E67734A
:10089000203120616E64203220617265206571759F
:1008A000616C00747279696E6720746F2072657371
:1008B000746F7265206C6173742072656164696E17
:1008C0006720666F72204300207374617274696ED2
:1008D000672E2E2E0073656E642064617461206F34
:1008E0006E206E6F496D70546F7574204300202820
:1008F0006E6F496D70546F75742900494E464F3ABA
:1009000020736176656420696D70436F756E742025
:1009100043002028666978656420696E7465727684
:10092000616C2900494E464F3A2073617665642018
:10093000696D70436F756E742043000000000023E2
:100940000026002900040404040404040402020232
:100950000202020303030303030102040810204000
:100960008001020408102001020408102000000089
:10097000080002010000030407000000000000005E
:1009800000494E464F3A20736176656420616C6C75
:100990002063757272656E7420646174612E00004C
:1009A000DF1B11241FBECFEFD8E0DEBFCDBF24E098
:1009B000A2E1B3E001C01D92A53DB207E1F713E04B
:1009C000A0E0B1E0E8E3FAE302C005900D92A231A5
:1009D000B107D9F714E0C1EDD4E004C02197FE01BE
:1009E0000E94F21CC03DD107C9F70E941D160C944D
:1009F0001A1D0C94000083E480937C0080917A009F
:100A0000806480937A0080917A0086FDFCCF80918B
:100A10007800909179000895AF92BF92CF92DF92C3
:100A2000EF92FF920F931F93CF93DF936C017B01A3
:100A30008B01040F151FEB015E01AE18BF08C01734
:100A4000D10759F06991D601ED91FC910190F081A7
:100A5000E02DC6010995892B79F7C501DF91CF916A
:100A60001F910F91FF90EF90DF90CF90BF90AF90CC
:100A70000895FC01538D448D252F30E0842F90E0A4
:100A8000821B930B541710F0CF9608950197089589
:100A9000FC01918D828D981761F0A28DAE0FBF2F52
:100AA000B11D5D968C91928D9F5F9F73928F90E0A8
:100AB00008958FEF9FEF0895FC01918D828D981717
:100AC00031F0828DE80FF11D858D90E008958FEF54
:100AD0009FEF0895FC01918D228D892F90E0805C1D
:100AE0009F4F821B91098F739927089586E394E0A5
:100AF0000E946A0521E0892B09F420E0822F0895E5
:100B0000FC01A48DA80FB92FB11DA35ABF4F2C9182
:100B1000848D90E001968F739927848FA689B78979
:100B20002C93A089B1898C91837080648C93938D70
:100B3000848D981306C00288F389E02D80818F7D13
:100B400080830895EF92FF920F931F93CF93DF93CB
:100B5000EC0181E0888F9B8D8C8D98131AC0E889F9
:100B6000F989808185FF15C09FB7F894EE89FF89C8
:100B70006083E889F98980818370806480839FBF66
:100B800081E090E0DF91CF911F910F91FF90EF9066
:100B90000895F62E0B8D10E00F5F1F4F0F73112776
:100BA000E02E8C8D8E110CC00FB607FCFACFE889B1
:100BB000F989808185FFF5CFCE010E948005F1CFB4
:100BC000EB8DEC0FFD2FF11DE35AFF4FF0829FB725
:100BD000F8940B8FEA89FB8980818062CFCF0F93D5
:100BE0001F93CF93DF938C01D0E0C0E0F801EC0FAE
:100BF000FD1F6491662341F086E394E00E94A20504
:100C0000892B11F02196F2CFCE01DF91CF911F9168
:100C10000F910895CF93DF93EC01888D8823B9F06D
:100C2000AA89BB89E889F9898C9185FD03C08081F7
:100C300086FD0DC00FB607FCF7CF8C9185FFF2CF74
:100C4000808185FFEDCFCE010E948005E9CFDF9145
:100C5000CF910895833081F028F4813099F082306B
:100C6000A9F008958730A9F08830C9F08430B1F434
:100C7000809180008F7D03C0809180008F7780936A
:100C80008000089584B58F7784BD089584B58F7DE5
:100C9000FBCF8091B0008F778093B0000895809152
:100CA000B0008F7DF9CFCF93DF9390E0FC01E75A3E
:100CB000F64F24918B5B964FFC0184918823C9F0F9
:100CC00090E0880F991FFC01E15CF94FA591B49168
:100CD000FC01EB5CF94FC591D49161110DC09FB738
:100CE000F8948C91209582238C93888128232883E3
:100CF0009FBFDF91CF910895623051F49FB7F89470
:100D00003C91822F809583238C93E8812E2BEFCF0B
:100D10008FB7F894EC912E2B2C938FBFEACF3FB76F
:100D2000F8948091ED039091EE03A091EF03B091C0
:100D3000F00326B5A89B05C02F3F19F00196A11D11
:100D4000B11D3FBFBA2FA92F982F8827BC01CD0115
:100D5000620F711D811D911D42E0660F771F881F74
:100D6000991F4A95D1F708958F929F92AF92BF92A3
:100D7000CF92DF92EF92FF926B017C010E948F066F
:100D80004B015C01C114D104E104F104B9F00E94EB
:100D90008F06681979098A099B09683E73408105A5
:100DA000910580F321E0C21AD108E108F10888EE2C
:100DB000880E83E0981EA11CB11CE4CFFF90EF9039
:100DC000DF90CF90BF90AF909F908F9008952FB7F6
:100DD000F8946091E9037091EA038091EB0390919C
:100DE000EC032FBF0895FC0101900020E9F7319733
:100DF000AF01481B590BBC0186E394E00C940C0531
:100E00008AE491E00C94F306CF93DF930E94EF0500
:100E1000EC010E9400078C0F9D1FDF91CF91089578
:100E20008F929F92AF92BF920F931F93CF93DF93B6
:100E3000CDB7DEB7A1970FB6F894DEBF0FBECDBF1A
:100E400019A2423008F44AE08E010F5D1F4F842E34
:100E5000912CB12CA12CA50194010E94D01CE62F4D
:100E6000B901CA01EA30F4F4E05DD801EE938D01D6
:100E7000232B242B252B79F790E080E0109719F095
:100E8000CD010E94F306A1960FB6F894DEBF0FBE07
:100E9000CDBFDF91CF911F910F91BF90AF909F90E9
:100EA0008F900895E95CE1CF009711F00C94F30660
:100EB00090E080E00895CF93DF930E94F306EC0169
:100EC0000E9400078C0F9D1FDF91CF910895BC01F8
:100ED00090E080E04AE00C941007CF93DF930E94EB
:100EE0006707EC010E9400078C0F9D1FDF91CF91D7
:100EF0000895CF92DF92EF92FF92CF93DF936C0130
:100F0000990FEE08FF08F7FE19C06DE286E394E042
:100F10000E94A205EC0166277727CB016C197D0999
:100F20008E099F094AE00E9410078C0F9D1FDF91D8
:100F3000CF91FF90EF90DF90CF9008954AE0C701E6
:100F4000B601DF91CF91FF90EF90DF90CF900C949E
:100F50001007CF93DF930E947907EC010E940007EE
:100F60008C0F9D1FDF91CF910895CF93DF93C82FF2
:100F70008DED90E00E94EF05D0E0CE0101960E9439
:100F800079078FEC90E00E94EF05CC0FDD1FFE018A
:100F9000E05FFE4F808191810E94670782EC90E0C4
:100FA0000E94EF05FE01E85FFE4F808191810E9463
:100FB000670787EB90E00E94EF05C45FDE4F8881F2
:100FC00099810E946707DF91CF910C940007682FE9
:100FD00070E090E080E04AE00C941007CF93DF933C
:100FE0000E94E707EC010E9400078C0F9D1FDF9114
:100FF000CF910895CF93DF934AE00E941007EC0150
:101000000E9400078C0F9D1FDF91CF9108958F9252
:101010009F92AF92BF92DF92EF92FF920F931F9336
:10102000CF93DF934A015B01D22EC82FD0E07E011F
:101030002FEFE21AF20A809100018E01000F111FBA
:10104000000F111FCC0FDD1F882309F47BC08DE832
:1010500090E00E94EF05C7010E94790780E890E0C8
:101060000E94EF05F801EF5EFB4F60817181828184
:1010700093814AE00E94100780E193E00E945407A8
:10108000FE01E05FFE4F808191818436910509F079
:1010900046C0FE01E75EFB4F808191810A9720F4F4
:1010A0008BEB91E00E945407FE01E75EFB4F8081CD
:1010B00091810E94670783E790E00E94EF05C05F7F
:1010C000DE4F888199810E946707DD2049F088E61C
:1010D00090E00E94EF054AE0C501B4010E941007AC
:1010E00080E591E00E945B07F801E750FC4F80919A
:1010F0000D0490910E04A0910F04B0911004808310
:101100009183A283B383DF91CF911F910F91FF90C1
:10111000EF90DF90BF90AF909F908F900895883EA2
:10112000934011F6FE01E75EFB4F808191818A308A
:10113000910518F48DE491E0B5CF8436910508F05F
:10114000B3CFAECF82E591E00E945407C7010E9461
:1011500079078DE592E00E945407F801EF5EFB4F9E
:1011600060817181828193814AE00E94100780E151
:1011700093E00E945407FE01E05FFE4F8081918161
:101180008436910551F5FE01E75EFB4F8081918128
:101190000A9720F48BEB91E00E945407FE01E75E72
:1011A000FB4F808191810E94670784E591E00E9456
:1011B0005407C05FDE4F888199810E946707DD2058
:1011C00049F084E591E00E9454074AE0C501B4016A
:1011D0000E9410070E94000787CF883E9340F1F6D7
:1011E000FE01E75EFB4F808191818A30910518F402
:1011F0008DE491E0D1CF8436910580F6CBCF20E00D
:1012000040E050E0BA0180E00E94070820E040E0A2
:1012100050E0BA0181E00C940708CF92DF92EF9280
:10122000FF920F931F93CF93DF93EB017B0124E099
:10123000E20EF11C8B016C01C61AD70AC601800FA1
:10124000911F0E94A41CF80181938F01EE15FF05E8
:10125000A9F7CE01DF91CF911F910F91FF90EF90F1
:10126000DF90CF9008950F931F93CF93DF938C015E
:10127000EB010E94A41C8883C80101960E94A41C53
:101280008983CE01DF91CF911F910F9108952F9205
:101290003F924F925F926F927F928F929F92AF9206
:1012A000BF92CF92DF92EF92FF920F931F93CF9353
:1012B000DF93CDB7DEB72E970FB6F894DEBF0FBE23
:1012C000CDBF362E1A8219821C821B829091070193
:1012D000482E512C911102C0662381F00E94000714
:1012E0000E9400078FEE91E00E94EF05C201019677
:1012F0000E9479078EE093E00E945B078201000F55
:10130000111FF801E25EFE4F808191819C878B87DF
:1013100096958795969587959A87898780910701F5
:10132000811102C0332061F086E591E00E945407EC
:1013300089859A850E946D078CEC91E00E940407D4
:10134000D12CC12C1E82B12CA12C712C612C212CF2
:101350001D8218861F82F801E65EFE4FFE87ED872C
:1013600089859A85C816D90608F0A7C04601880C59
:10137000991C880C991CED85FE85E080F180E80CB5
:10138000F91C80910701811102C03320B1F0C40122
:10139000969587959695879501960E94670781E6B1
:1013A00091E00E945407C4010E94670781E691E022
:1013B0000E945407C7010E946707C114D10421F09D
:1013C00089819A8198878F83BE016F5F7F4FC701A4
:1013D0000E943309BE016D5F7F4FC70102960E94D4
:1013E000330980910701811102C03320C1F081E6E9
:1013F00091E00E94540789819A810E94670783E6E1
:1014000091E00E9454078F8198850E94670783E6C8
:1014100091E00E9454078B819C810E946707E980BC
:10142000FA8080910701C114D104E9F4E114F104B8
:10143000D1F06B807C80811102C03320D9F185E628
:1014400091E00E94540791E09E83809107018111F1
:1014500001C031100E9400079FEFC91AD90A540138
:101460002E2CFD827DCF2F8138852F5F3F4F2E158B
:101470003F0579F4811102C0332021F085E691E027
:101480000E945407E980FA806B807C80E1E0EE8363
:10149000DCCFC984DA84FFEFCF1ADF0A811102C0E2
:1014A000332021F088E691E00E9454074501E22CA8
:1014B000FD80CBCF81E08E83C8CFEE81E11136C0B5
:1014C00080910701811127C0311025C0F801EF502C
:1014D000FC4F11821082F801EB50FC4F81E090E04C
:1014E000918380832E960FB6F894DEBF0FBECDBFDA
:1014F000DF91CF911F910F91FF90EF90DF90CF90F0
:10150000BF90AF909F908F907F906F905F904F9023
:101510003F902F9008958EE991E00E94EF05C2015F
:1015200001960E94A9073110DDCFD0CF7501F4E0FC
:10153000EF0EF11C8B859C8504978E159F0510F48A
:10154000F12CE12C8FE491E0311017C0F801EF503D
:10155000FC4FF182E082F801EB50FC4F20828D813C
:101560008183F801E75EFB4F71826082F801E75FDB
:10157000FB4F718260828AE791E00E94EF05C20111
:1015800001960E94790787E491E00E94EF05C3016C
:101590000E94670780910701811102C0332019F171
:1015A0008DE391E00E94EF05822D9D810E946707E7
:1015B00085E391E00E94EF05C50196958795969584
:1015C000879501960E9467078BE291E00E94EF05E4
:1015D000C5010E94670780E291E00E94EF05C70104
:1015E0000E946D077FCF0E9400077CCFCF93DF93CF
:1015F000EB010E94A41C8883CE01DF91CF91089556
:10160000FF920F931F93CF93DF93EC01F62E088187
:101610001981C8010E94A41CF81621F06F2DC80181
:101620000E94B21CCE01DF91CF911F910F91FF90CC
:1016300008950F931F93CF93DF9300D0CDB7DEB7FC
:101640008B019A838983FB016081CE0101960E9400
:10165000000BC8010F900F90DF91CF911F910F9158
:101660000895AF92BF92CF92DF92EF92FF920F93C5
:101670001F93CF93DF9300D0CDB7DEB78B016B0103
:1016800024E0C20ED11C7B015C01A61AB70AC50179
:101690008E0D9F1D9A838983F70161917F01CE0191
:1016A00001960E94000BEC14FD0489F7C8010F900D
:1016B0000F90DF91CF911F910F91FF90EF90DF90EE
:1016C000CF90BF90AF900895FF920F931F93CF9349
:1016D000DF93823008F048C0F62EC82FD0E08E018C
:1016E000000F111FC8018D5F9E4F0E94AC1C092E78
:1016F000000CAA0BBB0BFE01EE0FFF1FEE0FFF1F2E
:10170000EF5EFB4F408151816281738184179507A1
:10171000A607B70711F4FF2039F1CC0FDD1FCC0F5E
:10172000DD1FCF5EDB4FF801ED5FFE4FBE01808114
:1017300091810E94310BF801EC5BFE4FBE0180816C
:1017400091810E94310BF801E05CFE4FBE01808167
:1017500091810E94310B89EF90E0DF91CF911F9131
:101760000F91FF900C940407DF91CF911F910F917F
:10177000FF900895EF92FF920F931F93CF93DF9303
:1017800000D0CDB7DEB78C017B019A838983FB0142
:101790006081CE0101960E94000B0F5F1F4F1A83DC
:1017A0000983F7016181CE0101960E94000BC701F8
:1017B0000F900F90DF91CF911F910F91FF90EF90BD
:1017C0000895CF92DF92EF92FF920F931F93CF93E2
:1017D000DF93082F10E0E801CC0FDD1F61110EC070
:1017E000FE01E75FFB4F20813181FE01E75EFB4F89
:1017F000808191812817390709F49BC0FE01EB50C5
:10180000FC4F808191818F3F980709F09BC081E058
:1018100090E091838083FE01EF50FC4F1182108293
:10182000CE018F509C4F6C01FE01E65EFE4FE080C2
:10183000F180FC0180819181E80EF91E8091070101
:101840008823A9F18AE692E00E94EF05C80101967B
:101850000E94790782E692E00E94EF05FE01E75EB2
:10186000FB4F808191810E94670788E592E00E948A
:10187000EF05FE01EB50FC4F808191810E946707CC
:101880008EE492E00E94EF05F601808191810E9432
:10189000670786E492E00E94EF05F601808191815E
:1018A000969587959695879501960E946D07680194
:1018B000CC0CDD1CB601675E7B4FC70102960E940F
:1018C000BA0BB6016B507C4FC7010E94BA0B8BE17B
:1018D00092E00E940407FE01E75FFB4FDE01A75E76
:1018E000BB4F8D919C9191838083000F111F000F3E
:1018F000111FF801EF5FFB4F80910D0490910E04D2
:10190000A0910F04B091100480839183A283B383CC
:10191000FE01EF50FC4F808191810496C25EDE4F44
:1019200028813981245031092817390778F4118228
:101930001082DF91CF911F910F91FF90EF90DF9078
:10194000CF9008950196918380836ACF918380839D
:10195000F0CF60E080E00E94E10B60E080E00E9458
:10196000640B60E081E00E94E10B60E081E00E9496
:10197000640B81E899E00C940407CF93DF93EC01AA
:101980000E94A90C82E892E00E94EF05CE010E941D
:1019900079078BE691E00E945B0786E394E00E9462
:1019A0000A06E0914804F091490480818F7E80838B
:1019B000E0914804F09149048081877F8083E09121
:1019C0004804F091490480818F778083E091480436
:1019D000F091490480818F7D8083809150048093B1
:1019E0004F04BE01DD0F880B990B0E94B40661E025
:1019F00086E00E945306E3E7F9E08491EFE5F9E021
:101A0000D491EBE4F9E0C491CC2399F081110E94C8
:101A10002A06EC2FF0E0EE0FFF1FEB5CF94FA591CB
:101A2000B4918FB7F8949C91ED2FE095E923EC9356
:101A30008FBFDF91CF91089584EE90E00E9404075C
:101A40008091160190911701893C910530F466E16F
:101A500071E084E090E00E94BA0B809114019091B3
:101A60001501853F914030F464E171E086E090E03B
:101A70000E94BA0B80911801909119018115944030
:101A800030F468E171E088E090E00C94BA0B0895BE
:101A9000EF92FF920F931F93CF93DF9300D0CDB7B8
:101AA000DEB78C017C01E60EF71E81E0E81AF10832
:101AB00088E990E00E94EF05C8010E94790783E958
:101AC00090E00E94EF05C7010E94A907E016F10609
:101AD00074F080E193E00E9454071A83098360E068
:101AE000CE0101960E94000B0F5F1F4FEFCF81E7E1
:101AF00091E00E945B070F900F90DF91CF911F91B3
:101B00000F91FF90EF900895CF93DF938230B0F55F
:101B1000C82FD0E0CC0FDD1FFE01ED5FFE4F64E06B
:101B200070E0808191810E94480DFE01EC5BFE4FC8
:101B300064E070E0808191810E94480DFE01E05CCC
:101B4000FE4F64E070E0808191810E94480DFE01AB
:101B5000E25EFE4F60817181FE01E65EFE4F808194
:101B600091810E94480DFE01EF50FC4F11821082BE
:101B7000CB50DC4F81E090E099838883DF91CF9157
:101B800008952F923F924F925F926F927F928F9221
:101B90009F92AF92BF92CF92DF92EF92FF920F93FC
:101BA0001F93CF93DF93CDB7DEB766970FB6F89448
:101BB000DEBF0FBECDBF16EE212E13E0312E86E321
:101BC00094E00E946A05892B09F476C786E394E0C5
:101BD0000E9448052091E6033091E703F901E3599B
:101BE000FC4F80838D3019F08A3009F03DC7108298
:101BF000121613060CF02CC780910701882361F0A0
:101C000086E791E00E9454078DE693E00E94540716
:101C10008BE791E00E945B0742E050E06DE771E0E6
:101C20008DE693E00E940C1D892BB9F4EDE6F3E0FC
:101C300001900020E9F7E057F34079F480E891E063
:101C40000E94540781E991E00E94540784E991E0E1
:101C50000E9454070E94000742C04AE050E068E931
:101C600071E08DE693E00E940C1D892B09F046C0BF
:101C7000EDE6F3E001900020E9F7E857F340F1F5D5
:101C800085EB92E00E94040780EA92E00E9404073C
:101C900010E000E0F12CE12CC7010E94A41CD82E1A
:101CA0000115110539F4C7010E94790783E691E017
:101CB0000E9454078D2D0E94E70783E691E00E9461
:101CC00054075FEFE51AF50A07301105A4F00E94EA
:101CD000000710E000E0E11444E0F406E9F6109299
:101CE000E7031092E603EDE6F3E02E163F0609F453
:101CF00066CF1192FACF0F5F1F4FEDCF49E050E052
:101D000063EA71E08DE693E00E940C1D892B59F483
:101D1000EDE6F3E001900020E9F7E757F34019F40E
:101D20000E94A90CDCCF47E050E06DEA71E08DE63F
:101D300093E00E940C1D892BF1F4EDE6F3E0019095
:101D40000020E9F7E557F340B1F481E08093070103
:101D500021E030E03093020120930101898387E282
:101D600096E00E940407BE016F5F7F4F82E090E023
:101D70000E94190BB4CF47E050E065EB71E08DE6AF
:101D800093E00E940C1D892B91F4EDE6F3E00190A5
:101D90000020E9F7E557F34051F410920701109243
:101DA000020110920101198288E196E0DACF4AE03F
:101DB00050E06DEB71E08DE693E00E940C1D892BE5
:101DC000E9F5EDE6F3E001900020E9F7E857F3408C
:101DD000A9F560E072E080E890E00E94480D64E0C0
:101DE00070E080910301909104010E94480D64E02D
:101DF00070E084E290E00E94480D64E070E088E2C8
:101E000090E00E94480D60E870E080E892E00E9457
:101E1000480D64E070E080910501909106010E94F8
:101E2000480D64E070E080E390E00E94480D64E0BB
:101E300070E084E390E00E94480D51CF48E050E00C
:101E400068EC71E08DE693E00E940C1D892B41F552
:101E50008DE693E0DC010D900020E9F7CD018E5670
:101E6000934088309105E0F08830910529F481E0B5
:101E700096E00E94040733CF099709F030CF809194
:101E8000750389831A82CE0101960E940C1C815031
:101E9000823018F40E94840D22CF8AEE95E0E9CFBB
:101EA0004CE050E061ED71E08DE693E00E940C1D86
:101EB000892B59F4EDE6F3E001900020E9F7EA57A9
:101EC000F34019F40E94FF080ACF49E050E06EED9C
:101ED00071E08DE693E00E940C1D892B39F58DE6AB
:101EE00093E0FC0101900020E9F7CF018E5693406A
:101EF00089309105D8F08930910519F483ED95E08A
:101F0000B8CF0A9709F0EBCE8091760389831A82C5
:101F1000CE0101960E940C1C8150823020F461E0B9
:101F20000E944709DCCE8CEB95E0A3CF4BE050E05C
:101F300068EE71E08DE693E00E940C1D892BD9F4C8
:101F4000EDE6F3E001900020E9F7E957F34099F45A
:101F50008DEC92E00E94EF050E94FB040E9479073D
:101F600082EC92E00E94EF05809118019091190196
:101F70000E9467076FCE4BE050E064EF71E08DE6A2
:101F800093E00E940C1D892B09F064C08DE693E05C
:101F9000DC010D900020E9F7CD018E5693408D3085
:101FA000910508F457C0E3EFE80F90E080E08E174A
:101FB00074F48A35910548F4DC01A359BC4F1D9691
:101FC0002C91DC01AE5EBC4F2C930196F0CF0E2E0F
:101FD000000CFF0BEE5EFC4F10822DE0EDE6F3E00F
:101FE000DF010D900020E9F7BD016E56734083EFCD
:101FF000820F90E0422F50E04617570770F461E0DF
:1020000070E06C0F7D1F860F971F43595C4FDA01FC
:102010003C91DC013C932F5FE3CFE1E0F0E0EC0F7B
:10202000FD1F8E0F9F1FDC011C92CF010E940C1C14
:102030008C018AEA95E00E94EF05802F0E94E70755
:102040000E940007112710931901009318010E94A4
:102050001C0D45CE4AE050E060E072E08DE693E072
:102060000E940C1D892B89F4EDE6F3E0019000201D
:10207000E9F7E857F34049F4109200011982BE01D4
:102080006F5F7F4F83E090E073CE4AE050E06BE0FB
:1020900072E08DE693E00E940C1D892B69F4EDE659
:1020A000F3E001900020E9F7E857F34029F481E0DC
:1020B000809300018983E3CF48E050E066E172E05D
:1020C0008DE693E00E940C1D892BE1F58DE693E0EF
:1020D000DC010D900020E9F7CD018E569340089762
:1020E00088F180E093E00E94EF05809101019091DA
:1020F00002010E94790784EF92E00E94EF0580912F
:102100001601909117010E94790788EE92E00E94D3
:10211000EF0580911401909115010E9479078DEDD2
:1021200092E00E94EF0580911801909119010E94A0
:1021300067070E94000780E00E94B50781E00E94C7
:10214000B507CDCD4CE050E06FE172E08DE693E055
:102150000E940C1D892B09F0B3C08DE693E0FC01B1
:1021600001900020E9F7CF018E5693408E30910503
:1021700008F4A6C0E3EFE80F90E080E08E1774F457
:102180008A35910548F4DC01A359BC4F1D962C916A
:10219000DC01AE5EBC4F2C930196F0CF0E2E000CEE
:1021A000FF0BEE5EFC4F10829DE060E080E0ADE64C
:1021B000B3E0FD0101900020E9F7EE56F340262F31
:1021C00030E0492F50E04E175F07A8F443595C4FA9
:1021D000FA0140814C3269F0811109C0EBE0F0E076
:1021E000EC0FFD1F2E0F3F1FF90140836F5F9F5FB4
:1021F000E0CF892FFCCF4BE050E04C0F5D1F240F48
:10220000351FD9011C92882309F457C031E0380FDB
:10221000EDE6F3E0282F2095DF010D900020E9F78F
:10222000BD016E567340822F830F90E0432F50E024
:102230004617570770F461E070E06C0F7D1F860F42
:10224000971F43595C4FDA014C91DC014C933F5F7F
:10225000E3CFE1E0F0E0EC0FFD1F8E0F9F1FDC01EC
:102260001C92DD24D394CE010B960E940C1C8C0191
:10227000CE0101960E940C1C7C01B8ECB01760F0F6
:1022800087E995E00E94EF05802F0E94E70711275C
:102290001093170100931601DD2061F086E895E0A8
:1022A0000E94EF058E2D0E94E707FF24F092150192
:1022B000E09214010E940007CACE1982D12CD3CF1C
:1022C0004CE050E06CE272E08DE693E00E940C1D61
:1022D000892BE9F4EDE6F3E001900020E9F7EA57F5
:1022E000F340A9F48BE795E00E94EF058091160179
:1022F000909117010E94790789E392E00E945407A8
:1023000080911401909115010E94A907E8CC4AE040
:1023100050E06CE372E08DE693E00E940C1D892B87
:1023200009F0F4C08DE693E0DC010D900020E9F7A0
:10233000CD018E5693408A30910508F4E7C08A306B
:10234000910519F484E695E094CD8F30910508F459
:10235000C6CC8A5040E0082E000C990B242F30E0A8
:10236000281739076CF44A3548F4F901EE5EFC4F42
:1023700023593C4FD9011A962C9120834F5FEECF01
:102380008E5E9C4FFC01108287E492E00E9454070D
:1023900082E193E00E9454078BE791E00E945B0783
:1023A0008091120389831A82CE0101960E940C1C2F
:1023B000082F77247A94780EF1E0F71508F451C0CD
:1023C00088E592E00E945407802F0E94EE0782E188
:1023D00093E0DC010D900020E9F7CD01835193409B
:1023E000059708F446C06AE372E082E193E00E9438
:1023F000511C6C010150110B000F111FF801E45F1B
:10240000FE4F4F019801285F3E4F5901005F1E4F5C
:10241000C114D10409F463CC6DE370E0C6010E94DD
:10242000F81C009709F449C0DC011D927D01C6012A
:102430000E94561C6FE672E0C6010E94031D892BA4
:1024400019F58AE792E00E945407C7010E940C1C0C
:102450000E94A907C7010E940C1CF8019183808388
:1024600029C080911303803239F08DE495E00E94F9
:10247000040789E295E0FDCC8FE592E00E945407C5
:10248000802F0E94EE07F5CF66E872E0C6010E9439
:10249000031D892BD1F480E992E00E945407C70103
:1024A0000E940C1C0E94A907C7010E940C1CD501A8
:1024B0008D939C93872D0E94B50764E571E090E0B1
:1024C00080E00E94511C6C01A3CF6BE972E0C60151
:1024D0000E94031D892B71F483EA92E00E94540745
:1024E000C7010E940C1C0E94A907C7010E940C1C76
:1024F000F401B4CF89E395E00E94EF05C6010E9484
:1025000054078BE791E00E945B07D4CF49E050E08D
:102510006CEA72E08DE693E00E940C1D892B09F0B5
:10252000C0C0EDE6F3E001900020E9F7E757F34083
:1025300009F0B7C08BE195E00E94040750E1A52E99
:1025400051E0B52E64E3862E61E0962E7CE0C72E26
:1025500071E0D72EE8E36E2EE1E07E2EF8E0EF2E5C
:10256000F1E0FF2EACE34A2EA1E05A2E01E010E08C
:1025700087EF93E00E94EF05C8010E94790788EE7B
:1025800093E00E94EF05D5018D919C910E946D070B
:10259000F501808191818A30910539F08436910569
:1025A00021F0883E934009F058C0B501D2018D91C9
:1025B0009C910E94BA0B88EA93E00E94EF05C80143
:1025C0000E9479078AE993E00E94EF05F701808174
:1025D00091810E946D07D7018D919C9181319E4020
:1025E00008F047C0B701F301808191810E94BA0BC6
:1025F0008BE593E00E94EF05C8010E9479078DE406
:1026000093E00E94EF05D6018D919C910E946D0789
:10261000F6018081918181319E40B8F5B601D401E7
:102620008D919C910E94BA0BB2E0AB0EB11CE2E01E
:102630008E0E911CF2E0CF0ED11C22E0620E711CB6
:1026400032E0E30EF11C42E0440E511C0230110551
:1026500009F4FDCC02E010E08BCF8DED93E00E94F9
:10266000EF05C8010E94790781EB93E00E940407FF
:10267000A2CF8FE893E00E94EF05C8010E9479077E
:1026800084E693E00E940407B3CF82E493E00E94C3
:10269000EF05C8010E94790787E193E00E940407D3
:1026A000C3CF4BE050E066EB72E08DE693E00E9412
:1026B0000C1D892B09F043C14DE6E42E43E0F42EB6
:1026C000D7010D900020E9F7CD018E5693408B3055
:1026D000910508F434C10E9718F487EF94E0C9CB44
:1026E00080917803803209F0FACA809179038336A9
:1026F00009F0F5CA80917A038D8B1E8ACE0145962A
:102700000E940C1C082F1FEF180F89ED94E0123067
:1027100008F0AFCB8EEB94E00E94EF05802F0E9473
:10272000EE0782EC92E00E945B07F7010190002027
:10273000E9F7CF018E569340409708F4D0CA00E0E5
:10274000802F90E0FC01E359FC4F2785422F022E99
:10275000000C550B405351094A30510560F40930C3
:1027600040F44BE050E04C0F5D1F840F951FDC01DF
:102770002C930F5FE5CF322F3D7F3C3209F440C0F0
:10278000203209F040C0912C0F5FF12CEBE0F0E01B
:10279000EC0FFD1F8E0F9F1FDC011C92CF010E94CA
:1027A0002A1C2B013C01E0E0FF20B1F1911097CAF7
:1027B00081E394E00E94EF05C301B2010E94FA0791
:1027C000812F90E0FC01EE0FFF1FEE0FFF1FEF5E69
:1027D000FB4F4082518262827382880F991FFC01F5
:1027E000E75EFB4F11821082812F0E94840D61E011
:1027F000812F0E94640B61E0812F0E94E10B6FCA60
:1028000099249394C1CF21119BCF912CFF24F39451
:10281000BDCF8F7D09F42FC1A02FB0E0A359BC4FCD
:102820001F968C91282F082E000C330B2053310952
:102830002A30310570F7E93038F4A1E0B0E0AC0F90
:10284000BD1FAE0FB11D8C930F5FEF5FE5CFF5019C
:10285000E05FFE4F808191818A309105A1F4BAE05A
:10286000CB16D104B8F08AE794E00E94EF05F50199
:10287000E05FFE4F808191810E9467078EEC92E0BD
:102880000E945B072CCA84369105A9F5E4E6CE16B2
:10289000D10448F786EA94E00E94EF054AE0C301BC
:1028A000B2010E94100780E193E00E945407F501F5
:1028B000E05FFE4F808191818436910589F55AE071
:1028C000C516D10420F48BEB91E00E945407C60199
:1028D0000E946D07F701EE0FFF1FEE0FFF1FEF5E67
:1028E000FB4F4082518262827382F501E75EFB4FAB
:1028F000D182C08279CF883EF3E09F0731F428EE81
:10290000C21623E0D20630F2AECF8031974209F0F2
:10291000AACF40E1C41647E2D40608F0A4CFBACF4C
:10292000883E9340A1F67AE0C716D10418F48DE4EE
:1029300091E0CBCF84E6C816D10448F6C4CF4AE074
:1029400050E063ED72E08DE693E00E940C1D892B50
:1029500069F5EDE6F3E001900020E9F7E857F34070
:1029600029F588E294E00E94EF0581E090E00E9462
:1029700079078DE592E00E9454078091F5039091CC
:10298000F6030E946D0788E294E00E94EF0582E062
:1029900090E00E9479078DE592E00E9454078091B3
:1029A000F7039091F8030E946D0799C945E050E044
:1029B0006EED72E08DE693E00E940C1D892BE9F527
:1029C0008DE693E0DC010D900020E9F7CD018E56F5
:1029D00093408530910588F18530910529F490E088
:1029E00080E00E94BD0C7BC9EAEFE80F90E080E038
:1029F0008E1774F48A35910548F4DC01A359BC4F55
:102A000016962C91DC01AE5EBC4F2C930196F0CF54
:102A10000E2E000CFF0BEE5EFC4F108282E193E065
:102A20000E945B0782E193E00E940C1C8939BAE3A3
:102A30009B07B8F283E194E01CCA80E094E00E9416
:102A4000EF058DE693E00E9454078BE791E018CFE5
:102A50001092E7031092E603EDE6F3E02E163F0630
:102A600009F4ADC81192FACF2F5F3F4F3093E703BF
:102A70002093E603A4C821E030E02C0F3D1F2E0F69
:102A8000311DF9011082CE0101960E940C1C6C01CF
:102A9000E12EF12C5701AA0CBB1C9110D8CE82E676
:102AA00094E00E94EF05C301B2010E94FA0789E495
:102AB00094E00E94EF050BCF66960FB6F894DEBF48
:102AC0000FBECDBFDF91CF911F910F91FF90EF907F
:102AD000DF90CF90BF90AF909F908F907F906F903E
:102AE0005F904F903F902F9008950E94760581113E
:102AF0000C94C10D08951F920F920FB60F921124DE
:102B00002F933F934F935F936F937F938F939F93F5
:102B1000AF93BF93EF93FF9386E394E00E94800509
:102B2000FF91EF91BF91AF919F918F917F916F91A5
:102B30005F914F913F912F910F900FBE0F901F907B
:102B400018951F920F920FB60F9211242F938F9307
:102B50009F93EF93FF93E0914604F09147048081A7
:102B6000E0914C04F0914D0482FD1BC09081809156
:102B70004F048F5F8F7320915004821741F0E091D2
:102B80004F04F0E0EA5CFB4F958F80934F04FF9178
:102B9000EF919F918F912F910F900FBE0F901F90EB
:102BA00018958081F4CF1F920F920FB60F921124C7
:102BB0002F933F938F939F93AF93BF938091E9039C
:102BC0009091EA03A091EB03B091EC033091E803FC
:102BD00023E0230F2D3758F50196A11DB11D209339
:102BE000E8038093E9039093EA03A093EB03B09387
:102BF000EC038091ED039091EE03A091EF03B0916F
:102C0000F0030196A11DB11D8093ED039093EE0397
:102C1000A093EF03B093F003BF91AF919F918F9179
:102C20003F912F910F900FBE0F901F90189526E89F
:102C3000230F0296A11DB11DD2CFCF93DF93CDB745
:102C4000DEB764970FB6F894DEBF0FBECDBF7894A1
:102C500084B5826084BD84B5816084BD85B58260A1
:102C600085BD85B5816085BD80916E008160809352
:102C70006E001092810080918100826080938100BB
:102C800080918100816080938100809180008160CB
:102C9000809380008091B10084608093B100809126
:102CA000B00081608093B00080917A00846080934E
:102CB0007A0080917A00826080937A0080917A0015
:102CC000816080937A0080917A00806880937A0096
:102CD0001092C1000FB6F894A895809160008861A9
:102CE00080936000109260000FBE1092F603109265
:102CF000F5031092F2031092F10310921104109256
:102D00001204109213041092140410921D041092D5
:102D10001E0410921F041092200410922504109299
:102D2000F8031092F7031092F4031092F303109239
:102D300015041092160410921704109218041092A1
:102D40002104109222041092230410922404109261
:102D5000260460E086E00E94530662E082E00E9462
:102D6000530662E083E00E94530660ED77E080E066
:102D700090E00E94B40688E199E20FB6F894A89515
:102D8000809360000FBE90936000E0914604F09144
:102D9000470482E08083E0914604F091470410826A
:102DA000E0914204F09143041082E0914404F091D8
:102DB000450480E1808310924E04E0914A04F09132
:102DC0004B0486E08083E0914804F09149048081BF
:102DD00080618083E0914804F0914904808188609B
:102DE0008083E0914804F091490480818068808369
:102DF000E0914804F091490480818F7D808380E8D0
:102E000091E00E94540781E991E00E94540784E90F
:102E100091E00E94540788EC98E00E94EF050E9420
:102E200000071A8219828FEC97E00E940407BE0106
:102E30006B5F7F4F82E090E00E94F60A82EC97E0A1
:102E40000E94EF058D81823008F078C190E0909368
:102E50000201809301010E94790780910101909104
:102E60000201009709F063C1109207010E94000758
:102E7000BE016B5F7F4F83E090E00E94F60A83EA19
:102E800097E00E94EF058D81823008F063C10E94B7
:102E9000EE078D81813009F058C180930001BE0199
:102EA0006F5F7F4F84E090E00E9433098FE797E0E7
:102EB0000E94EF0589819A81893C910508F051C1F2
:102EC00090931701809316010E94A907BE016F5FBE
:102ED0007F4F86E090E00E9433098EE597E00E94E4
:102EE000EF0589819A81853F21E0920708F03EC174
:102EF00090931501809314010E94A907BE016F5F92
:102F00007F4F88E090E00E9433098FE397E00E94B2
:102F1000EF0589819A81811534E0930708F02BC170
:102F200090931901809318010E946D070E94000779
:102F300083E197E00E9404077CE3C72E71E0D72E5F
:102F4000E4E3AE2EE1E0BE2EF8E38F2EF1E09F2EFB
:102F5000A0E1EA2EA1E0FA2E01E010E00E940007B5
:102F600082E591E00E945407C8010E9479078CE62F
:102F700092E00E945407BE016F5F7F4FD6018D9192
:102F80009D916D010E94330987E097E00E94EF0553
:102F900089819A810E94670789819A818A30910587
:102FA00041F08436910529F0883EB3E09B0709F093
:102FB000EAC0F70191838083BE016F5F7F4FD40128
:102FC0008D919D914D010E94330980ED96E00E9404
:102FD000EF0589819A810E94670789819A818131F1
:102FE000BEE09B0708F0E8C0F801EE0FFF1FEA5FA4
:102FF000FE4F91838083BE016F5F7F4FF50181910A
:1030000091915F010E94330986E896E00E94EF05E6
:1030100089819A810E94670789819A818131FEE0C6
:103020009F0708F0E2C0F801EE0FFF1FE65FFE4FBA
:103030009183808322E0E20EF11C0230110509F039
:103040009FC00E94000793E0C92E91E0D92E24E48E
:10305000A22E21E0B22E30E4832E31E0932E01E146
:1030600014E0EE24E394F12C60E08FEF8E0D0E94CB
:103070004709BE01675F7F4FD6018D919D916D011C
:103080000E940D09BE016B5F7F4FF5018191919107
:103090005F010E940D09BE016F5F7F4FD4018D91CA
:1030A0009D914D010E940D0980910701882379F0BF
:1030B0000E9400070E94000783EA98E00E94EF0543
:1030C000C7010E9479078EE093E00E945B07898523
:1030D0009A85AB85BC854D815E816F8178854980FD
:1030E0005A806B807C8084179507A607B70709F084
:1030F000A3C0F80180839183A283B38384159505CF
:10310000A605B70509F08EC084EE97E00E94EF0592
:10311000C7010E9479078DE592E00E945407F801EB
:1031200060817181828193810E94FA07B1C0019709
:1031300009F09CCE81E08093070198CE0E94E707BA
:103140008AEA97E00E94040791CE8111A8CE1092DE
:103150000001A5CE0E94E7078BE897E00E940407D4
:103160009ECE8AE697E00E940407B0CE89E497E0FD
:103170000E940407C3CE8AE297E00E940407D6CEDD
:1031800002E010E0EBCE0E9400078CEF96E00E9478
:10319000EF05C8010E9479078DED96E00E940407B3
:1031A00082E591E00E945407C8010E9479078CE6ED
:1031B00092E00E94540700CF0E94000785EC96E041
:1031C0000E94EF05C8010E94790781E996E00E94FC
:1031D000040782E591E00E945407C8010E94790724
:1031E0008CE692E00E94540706CF0E9400078BE70E
:1031F00096E00E94EF05C8010E94790789E496E0F5
:103200000E94040782E591E00E945407C8010E94D1
:1032100079078CE692E00E9454070CCF82E0E82EFA
:10322000F12C22CF80910701882309F46DCF8BE721
:1032300098E00E94040768CF84159505A605B70598
:1032400069F4F80180839183A283B383809107019D
:10325000882309F459CF83E598E0EBCF4415550551
:103260006605770571F4D8014D935D936D937C935A
:10327000139780910701882309F446CF8BE298E0E9
:10328000D8CF80E098E00E94EF05C7010E94A9070F
:103290000C5F1F4FF2E0EF16F10409F0BFCF0E9460
:1032A000FF08332433940E94E70600913204109102
:1032B00033042091340430913504601B710B820B70
:1032C000930B683E73408105910508F452C10E943A
:1032D000E706609332047093330480933404909330
:1032E0003504B8E0EB2EB1E0FB2E19EF812E13E090
:1032F000912E49E154E05E874D8789E094E09C8BF4
:103300008B8B6C015A0110E000E0202ED7018D91CB
:103310009C91892B09F49EC0F60120813181D50151
:103320008D919C912817390709F478C00E94E7060F
:10333000F801EE0FFF1FEE0FFF1FE35EFB4F408013
:103340005180628073809B01AC01241935094609C4
:1033500057092F87388B498B5A8BD7012D913C9178
:10336000E8EEF3E02E9FC0012F9F900D3E9F900D41
:103370001124B0E0A0E04F84588869887A88481604
:1033800059066A067B0608F449C0D5018D919C91C7
:10339000F6019183808360E0802F0E94E10B8BEF28
:1033A00098E00E94EF05C80101960E9479078EEE11
:1033B00098E00E94EF050E94000780910701882392
:1033C000A9F085ED98E00E94EF05C80101960E94E2
:1033D000790784EE92E00E945407F7018081918181
:1033E0000E94670786EE92E00E945B0721E040E0C2
:1033F00050E0BA01822D0E94070880910D0490913F
:103400000E04A0910F04B0911004F4018083918305
:10341000A283B3831FC001E010E077CF40910D0479
:1034200050910E0460910F0470911004F40180819A
:103430009181A281B381481B590B6A0B7B0BD70189
:103440008D919C91B0E0A0E0481759076A077B076F
:1034500008F0B3CFF2E0EF0EF11C24E0820E911CD5
:1034600032E0A30EB11C42E0C40ED11C01301105A4
:1034700091F67CE0C72E71E0D72EE1E0EE2EE4E07D
:10348000FE2E10E000E0D6012D913D916D01211539
:10349000310509F448C0EB89FC8940815181AD8533
:1034A000BE858D919C9148175907E9F140910D0413
:1034B00050910E0460910F0470911004F701808107
:1034C0009181A281B381481B590B6A0B7B0BFCE3F2
:1034D000F29FC001F39F900D1124B0E0A0E04817C7
:1034E00059076A077B07F8F060E0802F0E94E10B24
:1034F00080910D0490910E04A0910F04B0911004DE
:10350000F70180839183A283B38384E299E00E94D0
:10351000EF05C80101960E94790782E199E00E94B7
:10352000EF050E9400072B893C892E5F3F4F3C8BA3
:103530002B8B4D855E854E5F5F4F5E874D8754E0D8
:10354000E50EF11C0130110509F088C080910D04D1
:1035500090910E04A0910F04B09110040196A11D4A
:10356000B11D80930D0490930E04A0930F04B093AB
:10357000100488E491E09E878D8757E2E52E54E0A1
:10358000F52E6FE2C62E64E0D62E10E000E0702E1D
:10359000AD85BE852D91BE87AD8730E0F901E35939
:1035A000F64F8491F901E75AF64FB490F901EB5BBD
:1035B000F64FA490AA2079F081110E942A06EA2DE4
:1035C000F0E0EE0FFF1FE55CF64FA591B491EC9192
:1035D000BE2281E009F480E0F60190818111BEC035
:1035E000913009F041C00E94E706D7016D937D93A9
:1035F0008D939C931397F801EB5DFB4F1082F601BE
:103600001082B4E0EB0EF11CEFEFCE1ADE0A0130AF
:10361000110539F58091180190911901892BA9F0B4
:10362000809131048111BAC00E94FB0420911801DD
:10363000309119018217930740F4309231040E94AF
:10364000A90C89EE92E00E945B07A8950E9476057E
:10365000882309F428CE0E94C10D25CE01E010E098
:1036600012CF01E010E093CF9111CBCF0E94E7067B
:10367000D7018D909D90AD90BC90AB01BC014819D5
:1036800059096A097B098091160190911701092E49
:10369000000CAA0BBB0B84179507A607B70708F009
:1036A000B0CFF801EB5DFB4F5F0180818111A9CFA5
:1036B0000E94E706D7016D937D938D939C9313979A
:1036C000F50130820E94E7062801440C551C440C89
:1036D000551CF201E35EFB4F80809180A280B38095
:1036E0009B01AC01281939094A095B0949015A01B2
:1036F0006083718382839383A801440F551FFA016D
:10370000E75EFB4F208131812F5F3F4F3183208364
:10371000405F5E4FDA014D915C9124173507B8F098
:10372000D201AF5EBB4F4D915D916D917C9113972E
:103730004F5F5F4F6F4F7F4F4D935D936D937C93C2
:1037400013971182108260E0872D0E94640B21E0A4
:10375000B501A401872D0E94070853CF911151CFC5
:103760000E94E706F7014080518062807380AB01C0
:10377000BC0144195509660977098091140190919B
:103780001501092E000CAA0BBB0B84179507A60781
:10379000B70708F036CFD6013C9233CF0E94FB0426
:1037A00020911801309119012C5E3F4F28173907DD
:1037B00008F04BCF1092310480E093E044CFE6E371
:1037C000F4E01382128288EE93E0A0E0B0E08483FC
:1037D0009583A683B78386E291E09183808385EC0D
:1037E00090E09587848784EC90E09787868780ECCB
:1037F00090E0918B808B81EC90E0938B828B82ECBC
:1038000090E0958B848B86EC90E0978B868B118E65
:10381000128E138E148E0895FC0188279927E89440
:1038200021912032E9F3293010F02E30C8F32B32E9
:1038300041F02D3239F4689404C00E949C1C820F20
:10384000911D219120532A30C0F31EF4909581954B
:103850009F4F08951F93FC0199278827BC01E89486
:1038600011911032E9F3193010F01E30C8F31B32F9
:1038700051F01D3249F4689406C00E94871C610F04
:10388000711D811D911D119110531A30B0F33EF43A
:1038900090958095709561957F4F8F4F9F4F1F91A9
:1038A000089543ED54E00E94601C0895DC016C9182
:1038B00061546A3108F060526F596D93C1F70895F1
:1038C000FA01A191B081009719F41097E1F0CD01B0
:1038D000DC01CD010D90002011F4C00113C0FB01EB
:1038E0002191222319F02015D9F7F3CFFB01219163
:1038F000201519F41E92119606C02223C1F70D90CF
:103900000020A1F7D001FA01A193B0830895592FA7
:10391000482F372F262F660F771F881F991F660F96
:10392000771F881F991F620F731F841F951F660FD3
:10393000771F881F991F08957AE0979F902D879F82
:10394000802D910D11240895F999FECF92BD81BD6E
:10395000F89A992780B50895A8E1B0E042E050E0D8
:103960000C94C21C262FF999FECF1FBA92BD81BDBF
:1039700020BD0FB6F894FA9AF99A0FBE01960895F1
:10398000DC01CB01FC01F999FECF06C0F2BDE1BD1F
:10399000F89A319600B40D9241505040B8F708950E
:1039A000A1E21A2EAA1BBB1BFD010DC0AA1FBB1F43
:1039B000EE1FFF1FA217B307E407F50720F0A21BB5
:1039C000B30BE40BF50B661F771F881F991F1A9422
:1039D00069F760957095809590959B01AC01BD014C
:1039E000CF010895EE0FFF1F0590F491E02D09948B
:1039F000FC018191861721F08823D9F79927089532
:103A00003197CF010895FB01DC018D910190801960
:103A10000110D9F3990B0895FB01DC01415050408E
:103A200030F08D910190801919F40020B9F7881BAE
:083A3000990B0895F894FFCFF3
:103A380001010020002C000100002C010F000000F3
:103A4800E803640046002800F401800080020002B8
:103A5800800000000000A2050C0539050A066A0569
:103A680048055C05120014000E0010000A000C0046
:103A7800280034002400300002030D0A0030300012
:103A88007D0043003B0064617461736574733A2080
:103A98000020200900095900094E006D732E2E2EB2
:103AA80000444F4E4500636D643A202700494400A6
:103AB8004475616C5330496D70436F756E746572EF
:103AC80000207600312E30006765742065657072BD
:103AD8006F6D00736176652064617461006465626E
:103AE80075672031006465627567203000666F7203
:103AF8006D617420616C6C00666F726D6174206317
:103B0800006765742072656164696E677300676534
:103B18007420696D70206300676574207077726720
:103B28006F6F640073657420707772676F6F6400DD
:103B3800736574206A736F6E203000736574206A31
:103B4800736F6E20310067657420636F6E66007353
:103B58006574206465626F756E63650067657420BF
:103B68006465626F756E6365002C20007365742050
:103B7800636F6E66206300636D64446174614275AF
:103B8800666665723A2027005F634E756D3D005F7B
:103B9800634E756D20696E76616C69643A200069C0
:103BA8006D70706572756E697400696D70506572BC
:103BB800556E69743D006E6F696D70746F75740031
:103BC8006E6F496D70546F75743D007361766569E9
:103BD8006E740073617665496E743D007361766535
:103BE80020636F6E66007365742072656164696E28
:103BF80067005345542052454144494E470020210F
:103C08002121006765742077636F756E7400726593
:103C1800736574002800732900504F574552204996
:103C28005320474F494E4720444F574E2E2E2E00C3
:103C3800504F57455220524553544F5245442E2E0B
:023C48002E004C
:00000001FF
